:020000040800F2
:100000000035002005010008D91500089B080008EC
:10001000D515000861080008411C00080000000018
:10002000000000000000000000000000AD19000802
:100030009908000800000000AD180008AF1900087A
:100040001F0100081F0100081F0100081F01000810
:100050001F0100081F0100081F0100081F01000800
:100060001F0100081F0100081F0100081F010008F0
:100070001F0100081F01000879080008890800080E
:100080001F0100081F0100081F0100081F010008D0
:100090001F0100081F0100081F0100081F010008C0
:1000A0001F010008A51A00081F0100081F01000811
:1000B0001F010008751B00081F0100081F01000830
:1000C0001F0100081F0100081F0100081F01000890
:1000D0001F010008311C00081F0100081F01000853
:1000E0001F0100081F0100081F010008DFF810D0E1
:1000F00000F0A4FB00480047FD2D0008AFF300808E
:10010000003500200648804706480047FEE7FEE726
:10011000FEE7FEE7FEE7FEE7FEE7FEE7FEE7FEE7B7
:10012000A11A0008ED000008D2B201E000F8012B8E
:10013000491EFBD270470022F6E710B513460A4667
:1001400004461946FFF7F0FF204610BD421C10F888
:10015000011B0029FBD1801A7047F0B480EA01022C
:10016000D40F4200B2EB410F02D2024608461146BC
:100170004A0042D0C30DDDB2C1F3C752AD1A202DE3
:1001800035DAC1F3160141F4000204B15242C5F15F
:10019000200602FA06F12A411044B3EBD05F23D0C7
:1001A000C4B1012DA0EBC35009DCF0BC4FF00042FC
:1001B00002EAC352DBB200F5000000F0B4BA40001E
:1001C00000F1807000EBC350A0F1807040EAD17064
:1001D000490009E0490841EAC071A0EBC35000F5AD
:1001E0000000400800EBC350F0BC00F093BA61423D
:1001F000012202EB4101001BF6E7F0BC704781F0E1
:100200000041AAE780F00040A7E780EA010210B5AC
:1002100002F00043400022D04A001FD0010E01EB43
:100220001261C0F35600C2F3560240F4000042F4DB
:100230000002A0FB022000047F39140400D0401CFF
:1002400050EA124001D44000491EC2B20C0604EB31
:10025000D010401C4008802A02D003E0002010BDCE
:1002600020F00100002900DA0020184310BD30B44E
:1002700080EA010202F0004530F0004221F0004027
:1002800013D090B1C30DD40DC2F31601C0F3160004
:10029000E41A41F4000140F400027D34914201D39C
:1002A000641C00E04900002C02DA30BC00207047DA
:1002B0004FF400000023914201D3891A0343400800
:1002C0004FEA4101F7D151B1914202D14FF00041C3
:1002D00005E002D24FF0010101E06FF0010103EBF4
:1002E000C450284430BC00F015BA2DE9FE4F8046BA
:1002F00081EA0300C00F0C46009021F0004123F07A
:100300000045B8EB0200A94105D24046214690467F
:100310001C460B46024623F00040104347D0270DF1
:10032000C7F30A00C3F30A510290401A0190402813
:100330006BDAC3F3130040F4801B0098924620B19F
:100340000023D2EB030A63EB0B0B01985946C0F173
:100350004002504600F0ADF906460D46504659465B
:10036000019A00F0C5F910EB08006141002487EA0A
:10037000115284EAE7731A4340D0009A62B3019A9B
:10038000012A4FEA075215DC001B61EB02014FF016
:10039000004202EA0752CDE90042001C41F58011FB
:1003A00032462B4600F0FCF903B0BDE8F08F404622
:1003B0002146F9E7001B61EB0201001C41F58013A7
:1003C00000185B412018A2F5001747EB030140EA33
:1003D000D570B6196D4111E06D084FEA360645EA51
:1003E000C0754FEA0752001B61EB0201001C41F58A
:1003F000801149084FEA30000019514132462B461E
:1004000003B0BDE8F04F00F0BCB9009801224000F5
:100410000023D0EB020263EBE073009821464FEA21
:10042000E074B8EB000061EB0401E9E783F00043FE
:100430005BE781F0004158E72DE9F04D81EA0304C4
:1004400004F0004B21F0004514464FF0000A23F061
:10045000004150EA050220D054EA01021DD0C5F344
:100460000A570246C5F31303C1F31300C1F30A563A
:1004700040F4801543F48013A7EB0608101BD64602
:1004800008F2FD3873EB050002D308F1010801E022
:1004900092185B41B8F1000F03DA00200146BDE875
:1004A000F08D00204FF48011064684460EE0171BA5
:1004B00073EB050705D3121B63EB050306434CEAF8
:1004C000010C49084FEA300092185B4150EA0107DD
:1004D000EDD152EA030012D082EA040083EA05015A
:1004E000084305D0101BAB4106D20122002306E0D1
:1004F00000224FF0004302E06FF0010253101AEBAC
:1005000006004CEB085110EB0A0041EB0B01BDE873
:10051000F04D00F036B9C10F80EAE0700844CA0718
:100520009623002100F0FFB896230022114600F028
:10053000FAB800F0004220F00040C10DC0F31600F0
:1005400040F400007F2901DA00207047962903DC7F
:10055000C1F19601C84001E096398840002AF4D0E4
:100560004042704720F00040C10DC0F3160040F437
:1005700000007F2901DA00207047962903DCC1F1D1
:100580009601C840704796398840704770B5C1F3EE
:100590000A5201F000450024C1F3130140F2FF3379
:1005A00041F480119A4201DA002070BD40F23343D9
:1005B0009A42A2F2334203DC524200F089F800E092
:1005C00090402C43F1D0404270BD00F0004230F02A
:1005D00000400AD0C10D01F56071C0F3160042EA77
:1005E0000151C2084007114370470020014670477F
:1005F00001F0004330B421F0004150EA010206D07E
:100600000A0DA2F56072C1F31301002A02DC30BCAE
:1006100000207047440F44EAC104C100E01830BC18
:1006200000EBC25000F076B8002801DBC0F10040BA
:10063000002901DBC1F1004181427047002801DB44
:10064000C0F10040002901DBC1F100418842704740
:100650002DE9F05F0546002092469B4688460646F7
:10066000814640241BE0284641464746224600F08A
:100670002FF853465A46C01A914110D311461846D6
:10068000224600F016F82D1A67EB01084F46224665
:100690000120002100F00DF817EB00094E41201E4B
:1006A000A4F10104DFDC484631462A464346BDE852
:1006B000F09F202A04DB203A00FA02F10020704764
:1006C0009140C2F1200320FA03F319439040704790
:1006D000202A04DB203A21FA02F00021704721FA97
:1006E00002F3D040C2F120029140084319467047FE
:1006F000202A06DBCB17203A41FA02F043EAE073E6
:1007000006E041FA02F3D040C2F1200291400843D2
:10071000194670470029A8BF7047401C490008BF10
:1007200020F00100704710B4B0FA80FC00FA0CF021
:1007300050EA010404BF10BC704749B1CCF1200459
:1007400021FA04F411FA0CF118BF012121430843E6
:10075000A3EB0C01CB1D4FEA00614FEA102042BF12
:10076000002010BC704700EBC35010440029A4BF08
:1007700010BC7047401C490008BF20F0010010BCAD
:10078000704710B5141E73F1000408DA401C41F1E3
:10079000000192185B411A4301D120F0010010BD05
:1007A0002DE9F04D92469B4611B1B1FA81F202E07B
:1007B000B0FA80F220329046FFF77BFF04460F46E6
:1007C00040EA0A0041EA0B0153465A46084313D057
:1007D000114653EA010019D0C8F140025046FFF714
:1007E00077FF05460E46504659464246FFF761FFE1
:1007F000084305D0012004E020463946BDE8F08DCD
:100800000020054346EAE0762C4337430A98630507
:10081000E40AA0EB08000022FD0A44EA47540A302B
:1008200002D500200146E9E7010510196941DDE91B
:10083000084500196941BDE8F04DA2E7064C074D97
:1008400006E0E06840F0010394E8070098471034A0
:10085000AC42F6D3FFF74EFC005A0008205A0008BD
:1008600000BFFEE7024600BF1AB901E000BF00BFAB
:10087000FCE700BF0120704710B50248006803F094
:1008800060FF10BD5C00002010B50248006803F056
:1008900058FF10BD5C000020704700BFFEE700005D
:1008A00008B5054989690143034A9161114689697F
:1008B0000140009100BF08BD0010024008B5054985
:1008C00089690143034A9161114689690140009198
:1008D00000BF08BD0010024008B505498969014301
:1008E000034A9161114689690140009100BF08BD2A
:1008F0000010024008B5054989690143034A916126
:10090000114689690140009100BF08BD00100240F6
:1009100010B54A1E044B9A5C825822F001034A1E0D
:10092000014CA25C835010BD384D000810B54A1E22
:10093000044B9A5C825842F001034A1E014CA25CAF
:10094000835010BD384D000810B54A1E044B9A5C08
:10095000825842F002034A1E014CA25C835010BD33
:10096000384D000830B54B1E054CE35CC35823F4EA
:10097000405313434C1E024D2C5D035130BD00000B
:10098000F64C000830B54B1E064CE35C03445B6834
:100990006FF30F0313434C1E024D2C5D0444636040
:1009A00030BD0000384D000830B54B1E054CE35CEF
:1009B000C35844F21004A34313434C1E014D2C5D55
:1009C000035130BDF64C000810B54B1E024CE35CE1
:1009D0000344DA6010BD0000384D000830B54B1EEE
:1009E000054CE35CC35823F0800313434C1E024DB7
:1009F0002C5D035130BD0000F64C000830B54B1E95
:100A0000054CE35CC35823F4406313434C1E024D72
:100A10002C5D035130BD0000F64C000830B54B1E74
:100A2000054CE35CC35823F0200313434C1E024DD6
:100A30002C5D035130BD0000F64C000810B54B1E74
:100A4000024CE35C03449A6010BD0000384D00087E
:100A500030B54B1E054CE35CC35823F040031343F1
:100A60004C1E024D2C5D035130BD0000F64C0008B9
:100A700030B54B1E054CE35CC35823F4407313435D
:100A80004C1E024D2C5D035130BD0000F64C000899
:100A90002DE9F04102460B461868C0F30F2595FA80
:100AA000A5F0B0FA80F480E00120A04028400028A2
:100AB0007AD0082C04D240F2011000FA04F106E0CA
:100AC000A4F108004FF00116864046F08061586896
:100AD00008280ED11869D66826EA11260F0A97FA57
:100AE000A7F7B7FA87F700FA07F73E43D66000BFCB
:100AF00000BF586802EB116691FAA1FCBCFA8CFCAD
:100B00004FEA8C084FF00F0C0CFA08FC376827EA04
:100B10000C0791FAA1FCBCFA8CFC4FEA8C0C00FA91
:100B20000CFC47EA0C07376000BF5868012802D068
:100B30005868092838D1986802EB116691FAA1FC2F
:100B4000BCFA8CFC4FEA8C084FF0030C0CFA08FC42
:100B5000376827EA0C0791FAA1FCBCFA8CFC4FEA33
:100B60008C0C00FA0CFC47EA0C07376000BFD86811
:100B700002EB116691FAA1FCBCFA8CFC4FEA8C08DE
:100B80004FF0040C0CFA08FC376827EA0C0791FABE
:100B9000A1FCBCFA8CFC4FEA8C0C00FA0CFC47EA76
:100BA0000C07376000BF00BF641C25FA04F0002862
:100BB0007FF47AAFBDE8F08102469068C1F30F235D
:100BC0001840C1F30F23984201D101207047002043
:100BD000FCE7C1F30F2242617047C1F30F2242616B
:100BE0007047C1F30F220261704770B500EB1163CB
:100BF00091FAA1F5B5FA85F5AE000F25B5401C6850
:100C0000AC4391FAA1F5B5FA85F5AD0002FA05F508
:100C10002C431C6070BD000002480068401C014964
:100C200008607047200000204FF47A71B0FBF1F2A9
:100C3000521E4FF0E0235A6100229A6105221A6188
:100C400000BF704710B5044600F066FE20602068C3
:100C500000F02EFE6060606800F03AFEA060606800
:100C600000F048FEE06010BD016841F04001016005
:100C7000704730B50246012300BF1068C0F38010F2
:100C800038BBD1E9000420438C682043CC68204362
:100C90000C6920434C6920438C692043CC69204374
:100CA0000C6A204314684FF6BF75AC4320431060B4
:100CB000506820F004004C6940EA14405060086A13
:100CC000B0F5005F04D1486A84B2146100BF00BF70
:100CD0000023184630BD000001490860704700003D
:100CE00000000020816821F080018160704701468A
:100CF000C86A704710B5024613681C48824208D083
:100D0000B2F1804F05D01A48824202D0194882427F
:100D100004D123F070004C6840EA04031348824277
:100D200008D0B2F1804F05D01148824202D011485C
:100D3000824204D123F44070CC6840EA040313607B
:100D40008868D06200BF0888906200BF074882426E
:100D500003D10869106300BF00BF00BF506940F0B5
:100D60000100506100BF002010BD0000002C0140B8
:100D7000000400400008004001460869C0F340003C
:100D8000704701460869C0F3800070470146086952
:100D9000C0F3C000704701460869C0F300107047F7
:100DA0000146086900F0010070470146C868C0F3B9
:100DB000400070470146C868C0F380007047014694
:100DC000C868C0F3C00070470146C868C0F300108F
:100DD00070470146C86800F00100704770B50246D0
:100DE000012901D1002416E0042901D1012412E0D7
:100DF000102901D102240EE0402901D103240AE088
:100E0000B1F5807F01D1042405E0B1F5806F01D1F7
:100E1000052400E006242346064CE55C02F1180494
:100E200028190468044DEE5C0425B540AC43046009
:100E300070BD0000D34C0008DA4C000870B50246C3
:100E4000012901D1002416E0042901D1012412E076
:100E5000102901D102240EE0402901D103240AE027
:100E6000B1F5807F01D1042405E0B1F5806F01D197
:100E7000052400E006242346064CE55C02F1180434
:100E800028190468044DEE5C0825B5402C43046025
:100E900070BD0000D34C0008DA4C00082DE9F04189
:100EA00006460C4615460127012C08D0102C0CD004
:100EB000B4F5807F0FD0B4F5805F18D111E02946DA
:100EC000304600F0CBFB074612E02946304600F0E2
:100ED00001FC07460CE02946304600F03DFC074681
:100EE00006E02946304600F073FC074600E000BFEC
:100EF00000BF3846BDE8F08181637047826844F2E4
:100F000007039A430A4382607047426822F07002E6
:100F10000A434260704708B50168009100BF41680C
:100F2000009100BF08BD6FF04001016070470000F4
:100F30002DE9FF4104460D4601270026204600F01A
:100F400055F8002833D1E9686868084329690843DF
:100F5000E16841F20C6291430843E060A8682169AE
:100F600021F440510143216100BF6869616921F4A6
:100F700040710143616100BF6846FFF763FE0E48A0
:100F8000844201D1039E08E00C48844201D1029EB4
:100F900003E00B48844200D1029E46B1286830B17C
:100FA0000027314620462A6800F025F800BF384661
:100FB00004B0BDE8F081000000380140004400406A
:100FC0000048004001460868C0F3400070470146F1
:100FD0000868C0F38000704701460868C0F3C0008D
:100FE000704701460868C0F3801070470146C86822
:100FF000C0F34030704770B501EBC10303EB011340
:101000009400B3FBF4F301EBC10404EB011495006D
:10101000B4FBF5F46425B4FBF5F404EBC40505EB6F
:101020000414A3EB8403322404EB03136424B3FB02
:10103000F4F303F0F00301EBC10404EB0114950099
:10104000B4FBF5F46425B4FBF5F403EB041401EBF5
:10105000C10303EB01139500B3FBF5F301EBC105ED
:1010600005EB01159600B5FBF6F56426B5FBF6F524
:1010700005EBC50606EB0515A3EB8503322505EB4D
:1010800003136425B3FBF5F303F00F0323449BB272
:10109000836070BD38B50120144949690143134A82
:1010A0005161114649690140009100BF00BF00F045
:1010B000FDFD05460022114600F090FA0446214647
:1010C0000E2000F003FE0E2000F0D6FD00F0EEFD35
:1010D00005460022114600F081FA044621460F2001
:1010E00000F0F4FD0F2000F0C7FD38BD00100240F5
:1010F00000B585B014216846FFF71DF81020FFF7F2
:10110000CFFB2020FFF7CCFB0420FFF7C9FB082012
:10111000FFF7C6FB2D492E48FFF75BFD41F618018E
:101120002C48FFF756FD2C492C48FFF752FD274865
:101130000090012001900220029000200390694657
:101140002348FFF7A5FC264800900020019069463F
:101150001F48FFF79DFC234800900020019069463E
:101160001C48FFF795FC41F6180000900120019003
:10117000022002900020039069461648FFF788FC81
:1011800040F20220009001200190022002900020F5
:10119000039069461148FFF77BFC1348009000203C
:1011A000019069460D48FFF773FC1048009001203C
:1011B00001900320029000200390012004906946D2
:1011C0000648FFF765FC05B000BD000020002004C4
:1011D000001001400008014032023004000C0140C0
:1011E000C000C0049F079904FFFCCF043000300406
:1011F00000B58FB0282105A8FEF79DFF1421684691
:10120000FEF799FF4FF48050FFF758FB0420FFF7DB
:1012100055FB4AF2A00000900920019001200290A5
:101220000020039069461348FFF732FC44F2400067
:1012300000900420019069460E48FFF729FC002029
:1012400005904FF4827006900020079002200890CD
:101250000120099040020A9018200B9000200C9069
:101260000D900A200E9005A90348FFF702FD0FB06C
:1012700000BD0000000801400030014030B585B0DD
:1012800014216846FEF757FF4FF40060FFF724FB78
:1012900000F014FD05460022032100F0BFF90446CA
:1012A0002146192000F026FD192000F0F2FC41F63D
:1012B0001F40ADF800000020019063200290002044
:1012C0000390049069460C48FFF714FD00BF0A48DC
:1012D000006820F080000849086000BF002106482F
:1012E000FFF70CFE00210448FFF70FFE0248FFF74E
:1012F000F9FC05B030BD0000002C014030B593B0C2
:1013000014210EA8FEF717FF202106A8FEF713FFF1
:10131000142101A8FEF70FFF02203249C9690143D9
:10132000304AD1611146C9690140009100BF00BF38
:1013300000F0C4FC05460022032100F06FF90446CA
:1013400021461D2000F0D6FC1D2000F0A2FC472005
:10135000ADF8380000200F904FF47A701090002004
:1013600011900EA92048FFF7C5FC00BF1E48006879
:1013700040F080001C49086000BF00211A48FFF7B8
:10138000BDFD4FF480711848FFF758FD60200690AE
:1013900000200790089009900A9006AA4FF48071E7
:1013A0001148FFF77BFD4FF480710F48FFF716FDE2
:1013B00000210D48FFF7A9FD0B48FFF793FC08201B
:1013C000FFF78AFA40F201100190092002900220F2
:1013D00003900020049001A90448FFF759FB13B0C3
:1013E00030BD00000010024000040040000C01402D
:1013F0002DE9F0418CB01C2105A8FEF79CFE1421BC
:101400006846FEF798FE4FF48040FFF773FA042019
:10141000FFF770FA684800900920019003200290BD
:101420000020039069466548FFF732FB644800904E
:101430000420019069466148FFF72AFB002205213C
:101440006048FFF7B1FA002205215E48FFF78AFAEB
:10145000002205215B48FFF7E1FA002205215948E7
:10146000FFF7F6FA802205215648FFF7B7FA002267
:1014700005215448FFF7FCFA002205215148FFF7E7
:10148000BDFA102204214F48FFF78EFA00220421F2
:101490004C48FFF767FA002204214A48FFF7BEFADA
:1014A000002204214748FFF7D3FA8022042145484F
:1014B000FFF794FA002204214248FFF7D9FA0022EC
:1014C00004214048FFF79AFA25213F4B1B68C3F3DC
:1014D0000220052400250346C3F1070CBCF1040FCC
:1014E00002D94FF0040C01E0C3F1070C674603F189
:1014F000040CBCF1070F02D24FF0000C01E0A3F185
:10150000030C66464FF0010C0CFA07FCACF1010C21
:101510000CEA040C0CFA06FC4FF0010808FA06F875
:10152000A8F1010808EA05084CEA080200BF0029F2
:1015300004DB1007030E2548435407E01007040E90
:1015400021480C3001F00F031B1FC45400BF25209D
:10155000002809DB00F01F0201219140420992009E
:1015600002F1E022C2F8001100BF4FF4E130059013
:1015700000200690079008900C20099000200A9007
:101580000B9005A91248FFF7D3FC00BF1048006973
:1015900020F490400E4908610846406920F02A0076
:1015A000486100BF00BF0846C06840F40050C860F2
:1015B00000BF0CB0BDE8F081020002040008014049
:1015C00004000404000002400CED00E000E400E030
:1015D0000038014000BFFEE700BFFEE7F0B503465C
:1015E0000C4603F00701C1F10700042801D90420CB
:1015F00001E0C1F107000646081D072801D20020BE
:1016000000E0C81E05460120B040401E2040A84012
:101610000127AF407F1E17403843F0BDF0B50346A9
:101620000C4603F00701C1F10700042801D904208A
:1016300001E0C1F107000646081D072801D200207D
:1016400000E0C81E05460120B040401E2040A840D2
:101650000127AF407F1E17403843F0BD70B50246EA
:10166000106A20F001001062136A5568946924F032
:10167000030424F070000E6840EA060423F0020020
:101680000E6940EA060323F001004E6840EA0603B3
:101690000F48824213D123F008004E6940EA8603C6
:1016A00023F004008E6840EA860325F480708E697A
:1016B00040EA060525F40070CE6940EA460555600B
:1016C0009461C868506300BF1362002070BD0000C1
:1016D000002C01402DE9F04104460D46206A20F01F
:1016E00010002062266AD4F80480A76927F44077A6
:1016F00027F4E040296840EA012726F02000296904
:1017000040EA011626F01000696840EA0116114807
:10171000844213D126F08000696940EA811626F0E0
:101720004000A96840EA811628F48060A96940EA6F
:10173000810828F40060E96940EAC108C4F804801F
:10174000A7612046E968FFF7D7FB26620020BDE8C5
:10175000F0810000002C014070B50246106A20F4B0
:1017600080701062136A5568D46924F0030424F071
:1017700070000E6840EA060423F400700E6940EA27
:10178000062323F480704E6840EA06230F48824205
:1017900013D123F400604E6940EA862323F480606D
:1017A0008E6840EA862325F480508E6940EA06154B
:1017B00025F40050CE6940EA46155560D461C868EA
:1017C000D06300BF1362002070BD0000002C0140F8
:1017D00070B50246106A20F480501062146A556891
:1017E000D36923F4407323F4E0400E6840EA0623F3
:1017F00024F400500E6940EA063424F480504E6808
:1018000040EA06340748824204D125F480408E69BC
:1018100040EA86155560D361C868106400BF146241
:10182000002070BD002C014070B5044600BFA06AC6
:10183000401C05490968B1FBF0F52046FFF757FA4F
:10184000401CB5FBF0F070BD000000202DE9F04118
:1018500005460E461746B0462846FFF748FA784335
:101860006421B0FBF1F084B2B8F1010F09D0B8F1F6
:10187000100F0AD0B8F5807F0BD0B8F5805F10D17B
:101880000BE000BF6C6300BF0CE000BFAC6300BFA7
:1018900008E000BFEC6300BF04E000BF2C6400BFA1
:1018A00000E000BF00BF00BFBDE8F081704700004E
:1018B000014600BF0448406800F0F0000009034AF8
:1018C000125C21FA02F0704700100240204D00081F
:1018D000014600BF0548406800F4E060044A02EB9E
:1018E0001020027821FA02F0704700000010024038
:1018F000304D0008014600BF0548406800F46050C4
:10190000044A02EBD020027821FA02F0704700006E
:1019100000100240304D000810B5002400BF0B48F5
:10192000406800F00C0020B1042804D0082808D139
:1019300003E0074C07E0064C05E000F00BF8044616
:1019400001E0034C00BF00BF204610BD0010024064
:1019500000127A000021002200BF1148406800F404
:10196000803002461AB1B2F5803F0CD101E00D493A
:101970000BE000BF0A484068C0F34040401C0A4BDF
:10198000B3FBF0F101E0074900BF00BF00BF04480E
:10199000406800F47010022303EB90404843704706
:1019A0000010024000093D0000127A0070477047A5
:1019B00010B502203749096821F007010143354A73
:1019C000116000BF00BF00BF3248006800F0070090
:1019D0000228F8D100BF3048006840F480302E491A
:1019E000086000BF00BF00BF2B480068C0F3404044
:1019F0000028F8D04FF480304FF4E011264A5268A6
:101A000022F47C1200F440330B431A43224B5A60F9
:101A100000BF00BF1846006840F08070194608609B
:101A200000BF00BF00BF1C480068C0F34060002832
:101A3000F8D000201849496821F0F0010143164A06
:101A4000516000BF10151146496821F4E06101435F
:101A5000516000BF00201146496821F460510143E4
:101A6000516000BF02201146496821F00301014383
:101A7000516000BF00BF00BF0748406800F00C0085
:101A80000828F8D10548FFF7CFF80448FFF724F9F4
:101A900010BD0000002002400010024000A24A04D5
:101AA0007047000010B53148FFF77AF901285CD182
:101AB00000BF2E48FFF760F901280AD12B48FFF735
:101AC00074F9012805D100BF001F2849086100BF33
:101AD00000BF2648FFF755F901280AD12348FFF730
:101AE00069F9012805D100BF801F2049086100BFA6
:101AF00000BF1E48FFF74AF901280BD11B48FFF72A
:101B00005EF9012806D100BF6FF00800174908618F
:101B100000BF00BF1548FFF73EF901280BD113485D
:101B2000FFF752F9012806D100BF6FF010000F49EE
:101B3000086100BF00BF0D48FFF732F901280AD144
:101B40000A48FFF746F9012805D100BFC01E074922
:101B5000086100BF00BF00BFFFF75EF800BF044888
:101B60000068401C0249086000BF10BD002C014005
:101B70005800002010B52D48FFF712F9012853D165
:101B800000BF2A48FFF7F8F801280AD12748FFF7D5
:101B90000CF9012805D100BF001F2449086100BFCE
:101BA00000BF2248FFF7EDF801280AD11F48FFF7D0
:101BB00001F9012805D100BF801F1C49086100BF41
:101BC00000BF1A48FFF7E2F801280BD11748FFF7CA
:101BD000F6F8012806D100BF6FF00800134908612C
:101BE00000BF00BF1148FFF7D6F801280BD10F48FE
:101BF000FFF7EAF8012806D100BF6FF010000B498B
:101C0000086100BF00BF0948FFF7CAF801280AD1E0
:101C10000648FFF7DEF8012805D100BFC01E0349C2
:101C2000086100BF00BF00BF10BD000000040040FD
:101C300010B50248006802F0AFFE10BD5C00002045
:101C400000BFFEE70FB47CB50C0009AD01D0611EEA
:101C500000E00021CDE90001064B6A4629460898BC
:101C600000F02AF9002C02D0009A002111707CBCEF
:101C70005DF814FB6D240008002809DB00F01F024A
:101C8000012191404209920002F1E022C2F80011C4
:101C90007047002809DB00F01F0201219140420932
:101CA000920002F1E022C2F8001170470248006879
:101CB000C0F30220704700000CED00E0024800680D
:101CC000C0F30220704700000CED00E010B50028C2
:101CD00004DB0A07130E054A135406E00A07140E24
:101CE000034A00F00F031B1FD45410BD00E400E0B2
:101CF00018ED00E010B5002804DB0A07130E054AB2
:101D0000135406E00A07140E034A00F00F031B1FCA
:101D1000D45410BD00E400E018ED00E002E008C873
:101D2000121F08C1002AFAD170477047002001E055
:101D300001C1121F002AFBD1704700002DE9F047B6
:101D400004460D4690461F46DDE908690CB10121A5
:101D500000E0002108468821FEF784FD0DB1012135
:101D600000E0002108468921FEF77CFDA16D09B144
:101D7000012100E0002108468A21FEF773FD656716
:101D8000C4F87880E667012084F8800084F8810038
:101D90000FB1C4F88470B9F1000F01D0C4F8889075
:101DA000A16D01F10C0000BF711E114A515C294464
:101DB000886000BF00BF0120686000BF00BF022034
:101DC000686000BF00BF701E1146085C285840F0D4
:101DD0000201701E105C295000BFA06D416841F0E7
:101DE0000201416000BFA06DFEF73EFFBDE8F08735
:101DF000624D0008014601F1100000E0001D02687C
:101E00001AB9024A12689042F8D370473400002091
:101E100070B504460D460CB1012100E000210846D2
:101E20007E21FEF71FFD0DB1012100E000210846D3
:101E30007F21FEF717FD002084F85C00A565284689
:101E4000FEF712FF70BD000010B50648046803E0FD
:101E50002046FFF7CFFF0446034800688442F7D3CB
:101E600010BD0000300000203400002010B50446F2
:101E70002146002001F0B6F810BD10B501E000F8D1
:101E8000011B131EA2F10104A2B2F8D110BD10B5BE
:101E900001E000F8011B131EA2F10104A2B2F8D167
:101EA00010BD10B501E000F8011B131EA2F10104E2
:101EB000A2B2F8D110BD00002DE9FF4F8DB00F4642
:101EC0000546002606E025280BD0DDE90F129047D5
:101ED0006D1C761C28780028F5D111B03046BDE87D
:101EE000F08F0024A246A1460122E94900E0044304
:101EF00015F8013F203B02FA03F00842F7D1287899
:101F00002A2810D06FF02F022878A0F1300109297B
:101F100014D80AEB8A0102EB410144F0020400EB01
:101F2000010A6D1CF0E701CF5FEA000A03D544F413
:101F30000054CAF1000A44F002046D1C28782E28CF
:101F400017D115F8010F44F004042A280ED06FF0C1
:101F50002F022878A0F1300109290AD809EB89015C
:101F600002EB410100EB01096D1CF2E757F8049BFD
:101F70006D1C28786C280FD006DC4C2817D06828F8
:101F80000DD06A2814D104E0742810D07A280FD11B
:101F90000DE044F400140AE044F4801401E044F439
:101FA00040146978814202D104F580146D1C6D1CC7
:101FB00028786E281ED00CDC632830D004DC002882
:101FC0008BD0582811D19FE0642867D069280CD1A4
:101FD00064E073282DD004DC6F2872D0702804D1FF
:101FE00094E075286ED078286DD0DDE90F12904707
:101FF000761C4BE1C4F30250022806D0032809D016
:10200000042801CF09D0066040E101CFF117C0E9F3
:1020100000613BE101CF068038E1067036E117F838
:10202000040B8DF8000000208DF80100EB46012024
:1020300003E057F804BB4FF0FF3061074FF0000199
:1020400002D40DE008F10101884649450FDA8045C8
:10205000F8DB1BF808100029F4D108E008F10101B1
:1020600088468142FADB1BF808100029F6D1DDE929
:102070000F23AAEB08008146214600F031F93044D5
:1020800000EB080604E0DDE90F121BF8010B904796
:10209000B8F10108F7D221464846F2E00A21C4F31C
:1020A00002524FF0000B0891022A04D001CFC11751
:1020B000032A09D00AE0FF1D27F00707F7E802010D
:1020C00008E02CE01EE01FE000B2C117042A01D195
:1020D00040B2C117021E71F1000206DA0023D0EBF4
:1020E000030063EB01012D2202E0220504D52B221F
:1020F0008DF82420012203E0E20701D02022F7E737
:10210000904653E00A210BE0102109E010214FF026
:10211000000B44F004044FF00809089103E0082183
:102120004FF0000B0891C4F30252022A04D001CFF1
:102130000021032A06D006E0FF1D27F00707F7E875
:10214000020103E080B2042A00D1C0B24FF00008BF
:1021500022072BD52A78702A07D0DDF820C08CF012
:10216000100C5CEA0B0C05D00EE040228DF8242008
:10217000012208E050EA010306D030238DF8243014
:102180008DF8252002229046089B83F0080353EA2D
:102190000B030BD150EA010201D1620706D53022B0
:1021A0008DF824204FF00108A9F101092A78582A56
:1021B00004D038A20B9208AA0A920BE03AA2F9E7DF
:1021C0005B46089AFEF744FA0B9B9B5C0A9A521EE8
:1021D0000A92137050EA0102F2D10A98ADEB0000A6
:1021E00000F1200B600702D524F4803401E04FF0A9
:1021F0000109D94502DDA9EB0B0000E0002000EB4E
:102200000B0141440890AAEB010AE00306D4DDE982
:102210000F232146504600F063F806444FF00009B2
:1022200008E009A911F80900DDE90F12904709F14A
:102230000109761CC145F4DBE0030CD5DDE90F2371
:102240002146504600F04CF8064404E0DDE90F1248
:1022500030209047761C0899481E08900029F5DC2C
:1022600008E00A980A990078491C0A91DDE90F12E2
:102270009047761CBBF10001ABF1010BF1DC21466C
:102280005046DDE90F2300F019F806446D1C21E6E5
:10229000092801003031323334353637383961623C
:1022A0006364656600000000303132333435363700
:1022B0003839414243444546000000002DE9F041D1
:1022C000044600251E461746880404D405E0394616
:1022D0002020B0476D1C641EF9D52846BDE8F0816A
:1022E0002DE9F041044600251E469046C80301D55D
:1022F000302700E02027880404D505E04146384611
:10230000B0476D1C641EF9D52846BDE8F0810FB4B6
:10231000DDE900108A68C0F30F231A40C0F30F23D1
:102320009A4201D1012200E00022D0B204B07047ED
:102330007CB504460CB1012100E000210846CF2104
:10234000FEF790FAA169D1E90401CDE90001A56980
:102350006E6995E80F00B0477CBD2DE9F047074650
:10236000884614461D464FF000090FB1012100E0D8
:1023700000210846FA21FEF775FA0CB1012100E0B0
:1023800000210846FB21FEF76DFA0DB1012100E0A6
:1023900000210846FC21FEF765FA384600F0EFFE02
:1023A0004146384600F0D9FF8146002606E0FF216D
:1023B000384600F0D2FFA055701CC6B2AE42F6DB24
:1023C000384600F0C1FE4846BDE8F0872DE9FC41E3
:1023D00004462169D1E90401CDE900012669F768C5
:1023E0003B4696E80700B84794F860102046226BF9
:1023F00090476620015D2046226B90470546216983
:10240000D1E90401CDE900012669D6E902733A4613
:10241000D6E90001B8472846BDE8FC8170B50446FE
:10242000002508E02846691C8DB244F620618842E8
:1024300000DD07E000BF2046FFF7C8FF00F0010005
:102440000028EFD100BF70BD0FB4DDE90001C1F37A
:102450000F22426100BF04B070470FB4DDE90001F4
:10246000C1F30F22026100BF04B070474A68002A1E
:1024700006D00A68531C0B6010704868401E486004
:10248000704710B504460CB1012100E00021084658
:10249000A321FEF7E7F9D4F8880018B12046D4F854
:1024A00088108847D4F8840018B12046D4F88410E6
:1024B000884710BDF0B50346002083F88100DC6F2B
:1024C000586F661E224FBE5D865926F00107661EB4
:1024D000DFF87CC01CF80660875100BFDC6F586FC6
:1024E000661E6746BE5D0644F16000BFDC6F586F34
:1024F000661EBE5D064476686FF30F061643671EC0
:102500001CF8077007447E6000BFDC6F586F661EC2
:102510006746BE5D865946F00107661E1CF80660D8
:10252000875100BF002507E0681C85B24CF250308F
:10253000854201DD00BF03E093F881000028F3D05D
:1025400000BF93F88100012800D1F0BD0020FCE716
:10255000624D000870B504460D4600260CB10121FD
:1025600000E00021084640F22911FEF77BF92046E1
:1025700000F005FE2946204600F0EFFE002120462F
:1025800000F0EBFE0646204600F0DEFD304670BD52
:102590002DE9FC4105460E4600270DB1012100E062
:1025A0000021084640F23D11FEF75CF92C460CB1C3
:1025B000012100E00021084640F2E221FEF752F935
:1025C000A169D1E90401CDE90001D4F818C0DCF813
:1025D0000C8043469CE80700C04700BF284600F037
:1025E000CEFD3146284600F0B8FE0746284600F0EA
:1025F000ABFD3846BDE8FC812DE9FC4705460E469B
:1026000017464FF000080DB1012100E000210846F7
:102610004FF4A871FEF726F92C460CB1012100E019
:102620000021084640F2D721FEF71CF9A169D1E943
:102630000401CDE90001D4F818C0DCE902934A4650
:10264000DCE90001C84700BF284600F098FD0024DF
:1026500007E03178284600F080FE8046761C601C3A
:1026600084B2BC42F5DB284600F06EFD4046BDE872
:10267000FC872DE9F04104460E46154600270CB1B3
:10268000012100E0002108464FF48A71FEF7EAF8C4
:10269000204600F074FD3146204600F05EFE0746FD
:1026A0002946204600F059FE204600F04DFD3846F0
:1026B000BDE8F0812DE9FC4105460E46012D01DA09
:1026C000012100E0002108468021FEF7CBF8C5EB90
:1026D0004510134901EB80040CB1012100E00021F9
:1026E00008468221FEF7BEF866B96168D1E90401A7
:1026F000CDE900016768D7F80CC0634697E807008A
:10270000E0470BE06168D1E90401CDE900016768A9
:10271000D7E902C36246D7E90001E047BDE8FC8182
:10272000803000202DE9FC4105460E46012D01DADE
:10273000012100E0002108466E21FEF793F8C5EB69
:102740004510214901EB80040CB1012100E000217A
:1027500008467021FEF786F8012E19D12168D1E9CB
:102760000401CDE900012768D7F80CC0634697E85B
:102770000700E04700BFA068016841F00101016067
:1027800000BFD4E90201026A0A43026200BF19E0F5
:102790002168D1E90401CDE900012768D7E902C326
:1027A0006246D7E90001E04700BFA068016821F058
:1027B0000101016000BFD4E90201026A8A4302629A
:1027C00000BF00BFBDE8FC81803000200FB430B5F1
:1027D000DDE90301C268C1F30F2323EA020402EA20
:1027E000030544EA0544046100BF30BC5DF814FBF6
:1027F0007CB504462169D1E90401CDE900012569D0
:10280000EE68334695E80700B0476320015D204637
:10281000226B90472169D1E90401CDE900012569C6
:10282000D5E902633246D5E90001B0477CBD7CB5ED
:1028300004462169D1E90401CDE900012569EE686A
:10284000334695E80700B0476220015D2046226BC1
:1028500090472169D1E90401CDE900012569D5E955
:1028600002633246D5E90001B0477CBD2DE9F04155
:1028700006460F4614461D464FF000080EB10121D2
:1028800000E000210846DE21FDF7ECFF0CB101213C
:1028900000E000210846DF21FDF7E4FF0DB1012132
:1028A00000E000210846E021FDF7DCFF304600F0A3
:1028B00066FC3946304600F050FD804604E0217841
:1028C000304600F04AFD641C281EA5F10101CDB27E
:1028D000F5D1304600F038FC4046BDE8F0810000FC
:1028E00010B516A1032001F09FF8C82000F0C0F831
:1028F00000F09CFF002405E0204601F03BF804F1C5
:102900000A00C4B2642CF7DD00200F4908600F49AB
:10291000086000BF00BF0E48006840F001000C498D
:10292000086000BF00BF0846C06840F00100C860F2
:1029300000BF00BF00F074FF10BD00004C4F4144C9
:10294000494E472E2E2E0000040000200C000020CF
:10295000002C014010B5034800F05EF8024800F07A
:10296000E1F910BD040000200C00002010B588B073
:1029700001F0E2FF01F0EBFA41F21001224800F011
:10298000BBF8059048F280011F4800F0B5F80290AE
:1029900042F220011C4800F0AFF8049044F24001DC
:1029A000194800F0A9F803900021084600F0A4F8A7
:1029B00006900021084600F09FF8079002A84FF407
:1029C0008073124A12490090002001F027FC40F663
:1029D00008010D4800F090F80446002001F00AFCC0
:1029E000046040F202210B4800F086F80446002003
:1029F00001F000FC4460002001F0FCFB012180F8A4
:102A0000641008B010BD0000000801400004004040
:102A100000300140000C014038B504460020009011
:102A2000206810B1112816D10BE000BF002001F082
:102A30008FFC00BF0A480068606000BF1120206062
:102A400000BF074960680968081A642801D200209D
:102A500038BD00BFEAE70020206000900320F7E7C0
:102A60005800002001490860704700001C00002049
:102A700070B504461E2094FBF0F594FBF0F100FBCA
:102A8000114604E047F2305000F012F86D1E002DA0
:102A9000F8D12EB14FF47A7106FB01F000F008F87E
:102AA00070BD00E000BF011EA0F10100FAD1704727
:102AB00070B5034600224FF0E02675690D4E36686A
:102AC00003FB06F44FF0E026B16910E04FF0E0267A
:102AD000B06988420BD0884202D20E1A324402E01A
:102AE0002E1A0E4432440146A24200D300E0EDE724
:102AF00000BF70BD1C0000202DE9F04105460E46C8
:102B000018273946002000F06DFA04460CB1012167
:102B100000E0002108463621FDF7A4FE256066602E
:102B20000548A0600548E0600548206105486061EF
:102B30002046BDE8F08100005B240008492400081D
:102B4000CD2700080F23000810B500BF01220E4951
:102B50000E48FEF74AF800BF0B490C48FEF741F853
:102B60000B490A48FEF73DF80420FFF7A1FF06498C
:102B70000648FEF732F80420FFF79AFF044903489D
:102B8000FEF72BF810BD000010001004000C0140EF
:102B90002000200410B500BF01220E490E48FEF7A8
:102BA00024F800BF0D490C48FEF717F809490A48F8
:102BB000FEF713F80420FFF77BFF08490648FEF7ED
:102BC00010F804490448FEF70CF80420FFF770FFE2
:102BD00010BD000010001004000C01402000200473
:102BE00010B50024082213491348FDF7FEFF1149D0
:102BF0001148FDF7F6FF0420FFF75AFF0F490E4872
:102C0000FDF7EFFF0420FFF753FF07E0601CC4B29D
:102C1000FA2C03DDFFF7BEFF002010BD0549064872
:102C2000FDF7CAFF0028F1D104490348FDF7D5FF9D
:102C30000120F2E710001004000C014020002004E5
:102C400070B50446002500BF012217491748FDF75B
:102C5000CCFF00BF16491548FDF7BFFF00BF1FE0BE
:102C6000E00920B110491148FDF7BBFF03E00E4910
:102C70000E48FDF7B2FF6006040E0220FFF718FFB2
:102C80000B490A48FDF7ADFF0220FFF711FF084985
:102C90000648FDF7A2FF0220FFF70AFF681CC5B235
:102CA000082DDDDB70BD000010001004000C014099
:102CB0002000200438B5044600208DF800008DF86F
:102CC0000140FFF741FF7820FFF7BAFFFFF788FFC9
:102CD0009DF80000FFF7B4FFFFF782FF9DF80100A9
:102CE000FFF7AEFFFFF77CFFFFF754FF38BD38B5A5
:102CF000044640208DF800008DF80140FFF724FFC6
:102D00007820FFF79DFFFFF76BFF9DF80000FFF7AE
:102D100097FFFFF765FF9DF80100FFF791FFFFF7B1
:102D20005FFF38BDF8B5044600200090206810B160
:102D30002B284DD142E000BF2848294BD968C0F369
:102D40000F2222EA010301EA020543EA0543244D6A
:102D50002B6100BF002001F097F922A20221002080
:102D600001F06CF8214908680968491C1F4B19607B
:102D7000FDF7DAFB054600232A460221282000F051
:102D800069FE1BA20421002001F058F8002001F088
:102D900031FA46693046FDF7C7FB054600232A464F
:102DA0000421282000F056FE01F026F900BF124849
:102DB0000068606000BF2B20206000BF0E49606883
:102DC0000968081A642801D20020F8BD00BFB3E7E3
:102DD0000020206000900320F7E70000200020047E
:102DE00000100140207469636B3A00001800002055
:102DF000206366673A0000005800002008B50120F3
:102E0000274989690143264A916111468969014030
:102E1000009100BF00BF00071146C9690143D1619D
:102E20001146C9690140009100BF00BF032002465E
:102E30001C4B19684FF6FF0319401B4B0B4343EA29
:102E40000221184B196000BF00BF1848406820F0ED
:102E5000E06040F000701549486000BFFEF7A8FD33
:102E6000134800681349B0FBF1F084B22046FFF725
:102E7000F9FDFEF73DF9FEF70DF9FEF7B9FAFEF799
:102E8000FDF9FEF73BFAFEF7B3F9002000F014F865
:102E9000FFF76CFDFFF724FD01E0FFF75BFDFCE7AA
:102EA000001002400CED00E00000FA0500000140B7
:102EB0000000002040420F0010B504460C4951F8B4
:102EC00024104A000B4951F82400002100F09EF81C
:102ED000094951F824200749083951F824000021F4
:102EE00000F094F8012103480830015510BD00009E
:102EF000A44D00084C000020B44D00082DE9F04717
:102F000004460F460025A9462348005D20B9224803
:102F100018380168204688471FB94FF0FF30BDE8D8
:102F2000F0871E4850F82400B7FBF0F61B4850F815
:102F30002400B7FBF0F100FB117000B1761C1848BB
:102F400050F82400451E22E01348083850F82400A9
:102F500030F8150010B909F1010901E04FF000093E
:102F6000B14513D14FF0000809E00B48083850F87C
:102F7000240005EB080220F8126008F10108B045B2
:102F8000F3D3064850F824006843C8E76D1E002DAF
:102F9000DADA4FF0FF30C2E754000020AC4D0008F1
:102FA000A44D000810B501460023002207E00B489D
:102FB00050F8210030F8120000B15B1C521C084888
:102FC00050F821009042F2D864205843044C54F841
:102FD0002140B0FBF4F0C0B210BD00004C00002056
:102FE000A44D000870B504460E4631462046FFF752
:102FF00085FF0546681C08B9002070BD024850F8DE
:1030000024002844F9E700004400002030B50346BE
:1030100001E003F8011B141EA2F10102F9D130BD39
:103020000FB42DE9F04105460D9F022D01DA012173
:1030300000E0002108463821FDF714FC90263146B7
:103040000020FFF7CFFF044600BF201D07A918226C
:1030500003E011F8013B00F8013B131EA2F1010649
:10306000B2B2F6D100BF67802570012084F85C0001
:103070002449A1642449E164244961652449216506
:10308000002D2ED12348E061234921622349A1620A
:103090002349E16223496162234921632349616332
:1030A0002349E1632349A1632349216423496164DE
:1030B000052084F86000012161200155062162206D
:1030C000015504216320015503216420015502218B
:1030D00065200155A521662001550021712001556B
:1030E0000AE0012D04D11648E0611649216203E08F
:1030F00061210020FDF7B6FB2046BDE8F0015DF838
:1031000014FB0000111E00083D1D0008B524000836
:103110008324000873260008552500086D28000840
:103120005B230008312300085B330008F5340008F6
:10313000E1310008DB350008E937000809330008F1
:1031400091250008F92500087CB504460CB1012141
:1031500000E00021084640F2ED21FDF783FB2169E4
:10316000D1E90401CDE900012569D5E902633246C0
:10317000D5E90001B047204600F01BF87CBD7CB5C6
:1031800004460CB1012100E00021084640F2F9217B
:10319000FDF768FB2169D1E90401CDE9000125694A
:1031A000EE68334695E80700B047204600F001F886
:1031B0007CBD70B5044600250CB1012100E0002162
:1031C000084640F26511FDF74DFB6588002D06DDD0
:1031D00000E000BF281EA5F101018DB2F9D170BD3C
:1031E0002DE9FC4704460D46174698464FF0010A64
:1031F00000260CB1012100E00021084640F2912197
:10320000FDF730FB0FB1012100E00021084640F23C
:103210009221FDF727FBB8F1000F01DD012100E04D
:103220000021084640F29321FDF71CFB2169D1E9FA
:103230000401CDE90001D4F810C0DCF80C904B4635
:103240009CE80700C8476420015D2046226B904738
:10325000064616B90020BDE8FC876720005D0228FD
:1032600010D1C5F307212046226B904706460EB9C0
:103270000020F0E7E9B22046226B9047064626BBC5
:103280000020E8E76720005D032819D1C5F3074156
:103290002046226B904706460EB90020DBE7C5F3B7
:1032A00007212046226B904706460EB90020D2E740
:1032B000E9B22046226B9047064636B90020CAE79D
:1032C0004FF42F710020FDF7CDFA4FF000090AE00E
:1032D0006620015D2046226B904707F8090009F13E
:1032E00001001FFA80F9C145F2DB2169D1E904012F
:1032F000CDE90001D4F810C0DCE902934A46DCE9CC
:103300000001C8475046A6E72DE9FC4104460D469A
:103310002169D1E90401CDE900012769D7F80CC082
:10332000634697E80700E04729462046226B90470E
:103330006620015D2046226B904706462169D1E94F
:103340000401CDE900012769D7E902C36246D7E944
:103350000001E0473046BDE8FC812DE9FC4704460A
:103360000D464FF0FF080CB1012100E00021084696
:1033700040F2B111FDF776FA94F85C0001287CD197
:10338000002795E026460EB1012100E00021084605
:1033900040F22631FDF766FAF168D1E90401CDE982
:1033A0000001D6F80CC0DCF80C904B469CE80700F6
:1033B000C84700BF2046FFF7FCFE05F08000C0B103
:1033C00026460EB1012100E00021084640F20531F9
:1033D000FDF748FA7168D1E90401CDE90001D6F89A
:1033E00004C0DCE902934A46DCE90001C84700BF9B
:1033F00018E026460EB1012100E0002108464FF4F6
:103400004471FDF72FFA7168D1E90401CDE900019B
:10341000D6F804C0DCF80C904B469CE80700C8477F
:1034200000BF00BF2046FFF7C4FE26460EB10121B3
:1034300000E00021084640F21B31FDF713FAF16865
:10344000D1E90401CDE90001D6F80CC0DCE9029312
:103450004A46DCE90001C84700BF2046FFF7A9FE45
:103460006806050E4FEA48604FEA1068A0680068D9
:10347000E0B1264616B1012101E01FE00021084617
:1034800040F23131FDF7EEF9B168D1E90401CDE93F
:103490000001D6F808C0DCF814909CE80F00C8477B
:1034A000012803D108F1010000F0FF08781CC7B221
:1034B000082FFFF667AF4046BDE8FC874FF0FF32AC
:1034C0000221204600F03FF808B9FF20F4E7A06D84
:1034D00000F10C010D7000BF4FF0FF3201212046BA
:1034E00000F031F808B9FF20E6E7A06D017B8846BF
:1034F0004046E1E77CB504460CB1012100E0002123
:10350000084640F2C921FDF7ADF92169D1E904016E
:10351000CDE900012569EE68334695E80700B0471C
:103520000A20FFF7BEFA2169D1E90401CDE90001C3
:103530002569D5E902633246D5E90001B0470A2082
:10354000FFF7AFFA7CBD2DE9F04104460D46164663
:1035500000270CB1012100E00021084640F2731160
:10356000FDF780F9022D0FD107E038467F1CB042ED
:1035700002D90020BDE8F08100BFA06D8168C1F3D1
:1035800040010029F1D026E0012D0ED106E0384699
:103590007F1CB04201D90020ECE700BFA06D81681C
:1035A00001F001010029F2D015E0802D0ED106E0D6
:1035B00038467F1CB04201D90020DBE700BFA06D78
:1035C0008168C1F3C0110029F2D004E04FF4D0713A
:1035D0000020FDF747F90120CCE72DE9FC5F044608
:1035E0000D46174698464FF0010A00260CB10121FE
:1035F00000E00021084640F20A21FDF733F90FB13F
:10360000012100E00021084640F20B21FDF72AF9D4
:10361000B8F1000F01DD012100E0002108464FF460
:103620000371FDF71FF9A16E09B1012100E000212E
:10363000084640F20D21FDF715F9D4F868902046B0
:10364000FFF7F5F82169D1E90401CDE90001D4F8CB
:1036500010C0DCF80CB05B469CE80700D84765203A
:10366000015D2046226B9047064616B90020BDE852
:10367000FC9F6720005D022810D1C5F3072120467A
:10368000226B904706460EB90020F0E7E9B22046CB
:10369000226B90470646DEB90020E8E7C5F30741F4
:1036A0002046226B904706460EB90020DFE7C5F39F
:1036B00007212046226B904706460EB90020D6E728
:1036C000E9B22046226B904706460EB90020CEE7AD
:1036D0006EE039782046226B904706460EB90020EE
:1036E000C5E77F1C7120005D002861D16D1CB5FB12
:1036F000F9F009FB105000285AD1B8F1000F57DD3E
:103700002169D1E90401CDE90001D4F810C0DCE958
:1037100002B35A46DCE90001D8472046FEF77EFE98
:103720002046FFF784F82169D1E90401CDE90001C1
:10373000D4F810C0DCF80CB05B469CE80700D84712
:103740006520015D2046226B904706460EB9002099
:103750008DE76720005D022810D1C5F307212046C0
:10376000226B904706460EB9002080E7E9B220465A
:10377000226B90470646DEB9002078E7C5F3074183
:103780002046226B904706460EB900206FE7C5F32E
:1037900007212046226B904706460EB9002066E7B7
:1037A000E9B22046226B904706460EB900205EE73C
:1037B000B8F10000A8F101011FFA81F889D121694F
:1037C000D1E90401CDE90001D4F810C0DCE902B36D
:1037D0005A46DCE90001D8472046FEF71FFE204686
:1037E000FFF706F8504642E770B504460D46164608
:1037F0000CB1012100E0002108464FF41F71FDF7D4
:1038000031F82046FFF713F8324629462046E3698F
:1038100098472046FEF702FE2046FEF7E9FF70BDFE
:1038200010B500F003F800F0E7FB10BD10B54FF441
:10383000806200210448FEF72AFB4FF48062FF21DA
:103840000248FEF724FB10BD80280020802C0020B9
:103850002DE9FC4F04460D4616461F46301B01D588
:10386000A01B00E0301B8146781B01D5E81B00E05F
:10387000781B8246B44201DA012001E04FF0FF30AC
:103880000190BD4201DA012001E04FF0FF300090CD
:10389000A9EB0A000FFA80F821E0294620460B9A8E
:1038A00000F022F8B44202D1BD4200D118E04FEA44
:1038B00048000FFA80FBCAF10000834506DDA8EB43
:1038C0000A000FFA80F801982044C4B2CB4506DA0A
:1038D00008EB09000FFA80F800982844C5B2DCE72D
:1038E00000BFBDE8FC8F0000F0B503461446802BF6
:1038F00001DA402900DBF0BD012C1CD1CD1701EB12
:103900005575ED1003EBC515194E755D0A46CE17BA
:1039100001EB5676F610A1EBC6070126BE403543F3
:10392000EEB20846CD1701EB5575ED1003EBC5154A
:103930000F4F7E551AE0CD1701EB5575ED1003EBD7
:10394000C5150B4E755D0A46CE1701EB5676F6107F
:10395000A1EBC6070126BE40B5430846CE1701EBD2
:103960005676F61003EBC616014FBD5500BFC2E7F1
:10397000802800203EB504460A25012005F11801E3
:103980000A236C220090184600F01CF801200090D9
:10399000201DC2B205F11A0107230C2000F0BCFA69
:1039A000234606A2052101A8FEF74CF901AA02212F
:1039B0002C2000F071FA00F01FFB3EBD253364257A
:1039C000250000002DE9F84104460D4616461F4625
:1039D000DDF81C80A019C2B22B4629462046CDF83E
:1039E0000080FFF735FFE819C3B2A019C2B2E81989
:1039F000C1B22046CDF80080FFF72AFFE819C3B214
:103A0000224629462046CDF80080FFF721FFE9191C
:103A1000CBB2A119CAB2A119C8B22946CDF800800B
:103A2000FFF716FFBDE8F88170B505460C46204645
:103A3000FCF78CFB00EB40008021A1EB4000C0F3C1
:103A4000470622462946304600F0F8F900F0D4FA3D
:103A500070BD00002DE9F04F87B005460E46914637
:103A60009A4600200390049005900290002483461B
:103A700000214846FCF7D8FD07D22D222046611CC4
:103A8000CCB203A90A5489F00049E3494846FCF73F
:103A9000D5FD02D207B0BDE8F08FC4F10800C0B276
:103AA0000290DE494846FCF7C9FD59D8DB49484633
:103AB000FCF7DDFB8046DA49FCF74FFB0746FCF7D5
:103AC00051FDC2B22046611CCCB203A90A5448463B
:103AD000FCF72FFD42F2107190FBF1F201FB120096
:103AE0004FF47A7190FBF1F03030C2B22046611C85
:103AF000CCB203A90A544846FCF71BFD4FF47A7177
:103B000090FBF1F201FB1200642190FBF1F03030E8
:103B1000C2B22046611CCCB203A90A544846FCF745
:103B200008FD642190FBF1F201FB12000A2190FBD9
:103B3000F1F03030C2B22046611CCCB203A90A5465
:103B40004846FCF7F6FC0A2190FBF1F201FB12005B
:103B50003030C2B22046611CCCB203A90A54C2E084
:103B6000B0494846FCF76AFD48D84846FCF7E1FCF6
:103B700042F2107190FBF1F201FB12004FF47A71E6
:103B800090FBF1F03030C2B22046611CCCB203A9E8
:103B90000A544846FCF7CDFC4FF47A7190FBF1F2E1
:103BA00001FB1200642190FBF1F03030C2B22046DC
:103BB000611CCCB203A90A544846FCF7BAFC642144
:103BC00090FBF1F201FB12000A2190FBF1F0303082
:103BD000C2B22046611CCCB203A90A544846FCF785
:103BE000A8FC0A2190FBF1F201FB12003030C2B2B6
:103BF0002046611CCCB203A90A5474E08A494846A5
:103C0000FCF71CFD34D84846FCF793FC4FF47A715E
:103C100090FBF1F201FB1200642190FBF1F03030D7
:103C2000C2B22046611CCCB203A90A544846FCF734
:103C300080FC642190FBF1F201FB12000A2190FB51
:103C4000F1F03030C2B22046611CCCB203A90A5454
:103C50004846FCF76EFC0A2190FBF1F201FB1200D2
:103C60003030C2B22046611CCCB203A90A543AE0FB
:103C70006E494846FCF7E2FC21D84846FCF759FC5F
:103C8000642190FBF1F201FB12000A2190FBF1F09C
:103C90003030C2B22046611CCCB203A90A54484657
:103CA000FCF747FC0A2190FBF1F201FB12003030D7
:103CB000C2B22046611CCCB203A90A5413E0002111
:103CC0004846FCF7BBFC0ED84846FCF732FC0A21FC
:103CD00090FBF1F201FB12003030C2B22046611CB1
:103CE000CCB203A90A54BAF1000F6ADD072C68DAD6
:103CF0002E222046611CCCB203A90A544846FCF788
:103D000018FC8046FCF707FC07464946FCF77AFAA0
:103D10008146BAF1010F1ED1082C1CDA43494846EE
:103D2000FCF773FA81464846FCF74FFC0022404BF3
:103D3000CDE90001FCF7D9FA0746FCF727FC0A2178
:103D400090FBF1F201FB12003030C2B22046611C40
:103D5000CCB203A90A54BAF1020F32DB082C30DAD4
:103D600031494846FCF751FA81464846FCF7E1FBE9
:103D7000642190FBF1F201FB12000A2190FBF1F0AB
:103D80003030C2B22046611CCCB203A90A54082CC0
:103D900017DA4846FCF719FC0022254BCDE9000153
:103DA000FCF7A3FA0746FCF7F1FB0A2190FBF1F2BE
:103DB00001FB12003030C2B22046611CCCB203A914
:103DC0000A5422E003A810F80B002038C0B2029079
:103DD000782D02DD0025701CC6B200240DE002988B
:103DE00000EB4000134901EB4000005D05EBC611FC
:103DF0002144114A5054601CC4B2062CEFDBA81DAC
:103E0000C5B20BF1010000F0FF0B03A810F80B0086
:103E10000028D7D100BF3DE60000FA4600401C460E
:103E20000000404200007A440000C84200002041E7
:103E30000000E03FE64D000880280020F0B5134662
:103E40000025002200241EE01E5D203EF5B27E28E3
:103E500002DD00204E1CF1B200220EE005EB45060B
:103E60000B4F07EB4606B65C00EBC1171744DFF8B3
:103E700024C00CF80760561CF2B2062AEEDB861D41
:103E8000F0B2661CF4B21E5D002EDDD1F0BD000064
:103E9000E64D000880280020F0B5034614460022B5
:103EA0000020002530E0665D203EF2B2782B02DD76
:103EB00000234E1CF1B200200CE000EB0216144F60
:103EC000BE5D03EBC1170744DFF848C00CF807607C
:103ED000461CF0B20828F0DB00200EE000EB0216D2
:103EE00008360B4FBF5D4E1C03EBC6160644DFF8C9
:103EF00024C00CF80670461CF0B20828EEDB03F173
:103F00000806F3B26E1CF5B2665D002ECBD1F0BD93
:103F10000E500008802800202DE9F84306460D4683
:103F200017469846DDF8209000240CE02819C3B20B
:103F3000F019C2B22819C1B23046CDF80090FFF78F
:103F400087FC601CC4B24445F0DBBDE8F88310B5C3
:103F5000AE20FEF7AFFE2020FEF7ACFE1020FEF7ED
:103F6000A9FEC820FEF7A6FE0020FEF7A3FE102043
:103F7000FEF7A0FE4020FEF79DFE8120FEF79AFE90
:103F8000FF20FEF797FEA120FEF794FEA620FEF785
:103F900091FEA820FEF78EFE3F20FEF78BFEA420A8
:103FA000FEF788FED320FEF785FE0020FEF782FE96
:103FB000D520FEF77FFEF020FEF77CFED920FEF72D
:103FC00079FE2220FEF776FEDA20FEF773FE12203D
:103FD000FEF770FEDB20FEF76DFE2020FEF76AFE86
:103FE0008D20FEF767FE1420FEF764FEAF20FEF77B
:103FF00061FEFFF715FC10BD70B500242DE0002612
:1040000000200DE000EBC4111D4A515C00EBC4120E
:104010001C4B9A5C914201D0012603E0411CC8B2BE
:104020008028EFDB00BFB6B104F1B001C8B2FEF7E3
:1040300041FE0120FEF73EFE1020FEF73BFE00256C
:1040400007E005EBC4110E4A505CFEF750FE681CF9
:10405000C5B2802DF5DB601CC4B2082CCFDB09484B
:1040600007494FF4806203E011F8013B00F8013B7F
:10407000131EA2F10104A2B2F6D100BF70BD000070
:1040800080280020802C00202DE9F0478146B9F1DE
:10409000010F01DA012100E000210846B821FCF7F8
:1040A000E1FBC9EB4910244901EB80040CB101216B
:1040B00000E000210846BA21FCF7D4FB0021484665
:1040C00000F004FA20636C21484600F0FFF96064B8
:1040D0000A21484600F0FAF9A0630B21484600F097
:1040E000F5F9E0631021484600F0F0F920647021F2
:1040F000484600F0EBF9A0640121484600F0E6F9DB
:1041000060635121484600F0E1F9A4F87400B4F866
:104110007410A1F2F670FCF7FEF98246FCF755FA2E
:104120000746064A064BFCF787F90546FCF760FA96
:10413000A067BDE8F087000080300020CDCCCCCC5B
:10414000CCCC1E4070B50546012D01DA012100E0FE
:10415000002108465521FCF785FBC5EB4510214998
:1041600001EB80040CB1012100E000210846572139
:10417000FCF778FB002060611B49A162A06A20F077
:10418000706000F1A060A0622121E1610021216244
:10419000164961621649E1620721A16100212846A2
:1041A000626900F0D3F96C212846A26A00F0CEF9CA
:1041B0000A212846E26900F0C9F90B212846226A43
:1041C00000F0C4F910212846626A00F0BFF970219E
:1041D0002846E26A00F0BAF901212846A26900F0F7
:1041E000B5F970BD80300020530141001F1F07004A
:1041F0001E264CC410B50446012C01DA012100E052
:1042000000210846A921FCF72DFBC4EB441002490C
:1042100001EB800010BD0000803000202DE9FF4739
:104220000546894616461F46DDF83080012D01DA25
:10423000012100E0002108469021FCF713FBC5EBAB
:104240004510284901EB8004A660E7600020039038
:10425000D8E90412D8F80C008DE80700002098E88F
:104260000E00FEF7DDFE2061216909B1012100E0A9
:10427000002108469521FCF7F5FA1C22002104F1E3
:104280001400FDF70EFE1C22002104F13000FDF7A2
:1042900008FE20694946826C9047134800684FF435
:1042A0007A71B0FBF1F06065A068816AA165A068D1
:1042B000FCF71DFD81B25C200153A068FDF7B4FA44
:1042C00020660A49A16600216C2001532167002065
:1042D00084F86400652001552846FFF733FFBDE8E8
:1042E000FF870000803000200000002000004842CE
:1042F0002DE9F04105460E46012D01DA012100E0CD
:1043000000210846AF21FCF7ADFAC5EB45100F4977
:1043100001EB80040CB1012100E000210846B1212D
:10432000FCF7A0FA00213046FCF77EF902D286F0B5
:10433000004000E030468046FCF714F987B23A4668
:10434000D4E90201FDF782FABDE8F0818030002057
:1043500070B50546012D01DA012100E00021084673
:10436000C921FCF77FFAC5EB4510194901EB800420
:104370000CB1012100E000210846CB21FCF772FAC4
:1043800094F864102846FEF7CDF96520015D2846B3
:10439000FEF790F9A068FCF7AAFC6C21095B884243
:1043A00010D06C20005B18B95C20015B6C200153BD
:1043B0006C22125B511EA068C16200BFA068FDF7AD
:1043C00033FA20672846A16EFFF792FF70BD000008
:1043D000803000202DE9FC4106460F469046012E14
:1043E00001DA012100E0002108461621FCF73AFA23
:1043F000C6EB4610344901EB80040CB1012100E00A
:10440000002108461821FCF72DFA216909B1012184
:1044100000E0002108461921FCF724FA206901690F
:10442000D1E90401CDE9000120690569D5F80CC086
:10443000634695E80700E047002507E0795D2069BD
:10444000026B904708F80500681C85B2052DF5DB66
:1044500020690169D1E90401CDE9000120690569FC
:10446000D5E902C36246D5E90001E04700BF00BFBD
:1044700000BF20690169D1E90401CDE9000120698B
:104480000569D5F80CC0634695E80700E0470025AC
:1044900007E0795D2069026B904708F80500681C09
:1044A00085B2052DF5DB20690169D1E90401CDE96B
:1044B000000120690569D5E902C36246D5E900011A
:1044C000E047BDE8FC810000803000207FB5044655
:1044D0000E46012C01DA012100E0002108464021AE
:1044E000FCF7C0F9C4EB4410174901EB80050DB18E
:1044F000012100E0002108464221FCF7B3F92969B7
:1045000009B1012100E0002108464321FCF7AAF986
:10451000002002900390009001908DF808606A4698
:1045200002A92046FFF756FF9DF8010000069DF8FE
:10453000021040EA01409DF8031040EA01209DF876
:104540000410084304B070BD803000202DE9FC4108
:1045500005460F461446012D01DA012100E0002135
:1045600008463021FCF77EF9C5EB4510164901EBF2
:1045700080060EB1012100E0002108463221FCF73F
:1045800071F9316909B1012100E0002108463321A8
:10459000FCF768F900200090019047F080008DF84A
:1045A0000000200E8DF80100200C8DF80200200A7A
:1045B0008DF80300E0B28DF804006946284600F04B
:1045C00005F8BDE8FC810000803000202DE9FC41A9
:1045D00005460F46012D01DA012100E000210846C1
:1045E0000721FCF73FF9C5EB45101E4901EB80049C
:1045F0000CB1012100E0002108460921FCF732F945
:10460000216909B1012100E0002108460A21FCF7D7
:1046100029F920690169D1E90401CDE90001206986
:104620000669D6F80CC0634696E80700E047002606
:1046300005E0B95D2069026B9047701C86B2052EBB
:10464000F7DB20690169D1E90401CDE900012069A6
:104650000669D6E902C36246D6E90001E047BDE833
:10466000FC8100008030002010B5044604B910BD64
:1046700000202085A07D012808D1606A30B1218CFE
:1046800089040A0C0021606AFDF7F7FB00BFEEE722
:104690002DE9F05F0646884615469946DDE90B7B15
:1046A000DDF828A00EB1012100E0002108462921F3
:1046B000FCF7D8F84420FDF7D9FB04460CB10121E2
:1046C00000E0002108462C21FCF7CCF80120E07521
:1046D00000202076C4F83C902584C4F840B0A7861A
:1046E000002D0CDD2846FDF7C1FBE061E16909B151
:1046F000012100E0002108463E21FCF7B3F8002F1D
:104700000CDD3846FDF7B2FB2063216B09B10121B6
:1047100000E0002108464521FCF7A4F884F8158044
:1047200084F82CA066602046BDE8F09F10B50446D2
:1047300004B910BD002060852046FFF795FF00BF3B
:10474000F7E710B504460CB1012100E0002108464E
:1047500040F2D711FCF786F8012084F8380021696F
:10476000A068FCF7D5F82069082865D2DFE800F0DA
:104770006404111E2C3A485600BFA0680168C1F3BA
:10478000400121B1A0680221416000BF00BF00BF0D
:1047900053E000BFA0680168C1F3401121B1A068D7
:1047A0002021416000BF00BF00BF46E000BFA068FD
:1047B0000168C1F3402129B1A0684FF40071416044
:1047C00000BF00BF00BF38E000BFA0680168C1F3B0
:1047D000403129B1A0684FF40051416000BF00BFD3
:1047E00000BF2AE000BFA0680168C1F3404129B1C1
:1047F000A0684FF40031416000BF00BF00BF1CE063
:1048000000BFA0680168C1F3405129B1A0684FF40E
:104810000011416000BF00BF00BF0EE000BFA068F4
:104820000168C1F3406129B1A0684FF00071416097
:1048300000BF00BF00BF00E000BF00BF606800BF56
:1048400000BF00BF00F10C0252E8002F42F040010F
:1048500000F10C0242E80013002BF3D100BF00BFAF
:104860002069082865D2DFE800F06404111E2C3AA4
:10487000485600BFA0680168C1F3C00121B1A0681B
:104880000821416000BF00BF00BF53E000BFA06827
:104890000168C1F3C01121B1A0688021416000BF4F
:1048A00000BF00BF46E000BFA0680168C1F3C0219F
:1048B00029B1A0684FF40061416000BF00BF00BF94
:1048C00038E000BFA0680168C1F3C03129B1A06819
:1048D0004FF40041416000BF00BF00BF2AE000BFAD
:1048E000A0680168C1F3C04129B1A0684FF400215C
:1048F000416000BF00BF00BF1CE000BFA0680168AE
:10490000C1F3C05129B1A0684FF40001416000BF5C
:1049100000BF00BF0EE000BFA0680168C1F3C06126
:1049200029B1A0684FF00061416000BF00BF00BF27
:1049300000E000BF00BF10BD0EB51348006808BB03
:104940000020F0210122114BCDE9002102900A46FE
:1049500001210F48FFF79CFE0B4908600020096801
:1049600008700C48084909688860052006490968EC
:10497000C8600420044909680861002102480068F1
:1049800000F0E2F80EBD00005C000020CB4C0008F7
:10499000003801400000024038B5044604B938BD73
:1049A0006068C168C1F34011B9B160680168C1F3C2
:1049B000401191B1608D218C884202DB2046FFF7C7
:1049C000B5FE61684A68D2B2608D411C6185E169BB
:1049D0000A5400202076E0753FE06068C168C1F3AA
:1049E0000011002939D060680168C1F30011002965
:1049F00033D0607D01282BD1D4E902014A1E514BEE
:104A00009A5C02445268208C801A6085207DF8B937
:104A1000D4E90201FBF77CFFE06B80B1608D0028D8
:104A20000DDD608D218C884209DC628D2078E36B7E
:104A3000E1699847228C0021E069FDF71EFA228C7B
:104A4000D4E90201FBF79EFFD4E90201FBF76EFFF8
:104A5000002060856068FCF75EFA6068C168C1F399
:104A6000801151B16068FCF7BCFA30B1206C08B11C
:104A7000206C80476068FCF756FAA07D01285ED163
:104A800001256068C168C1F3002171B160680168E7
:104A900001F0010149B1022560680168009100BF81
:104AA0004168009100BF00BF00BF6068FCF78AFA50
:104AB00068B16068FCF786FA48B10425606801684F
:104AC000009100BF4168009100BF00BF00BF606857
:104AD000FCF77DFA60B16068FCF779FA40B1606874
:104AE0000168009100BF4168009100BF00BF00BF96
:104AF0006068FCF771FA68B16068FCF76DFA48B15C
:104B0000102560680168009100BF4168009100BFF6
:104B100000BF00BF012D11D0606A78B1618D491EC0
:104B200088B2228D616A01EB82014880228D616A20
:104B300001F82250218D491C218500BF00BF00BF14
:104B40002DE70000384D000870B504460D46607D25
:104B500090B9A575606800BF00BF00BF00F10C02EE
:104B600052E8002F42F0200100F10C0242E800134D
:104B7000002BF3D100BF70E00020A0756068FCF747
:104B8000CAF92169A068FBF7C3FED4E90201FBF76B
:104B9000BFFE6068011D0E463246D4E90201FBF7F4
:104BA0004DFFE269D4E90201FBF70EFF228CD4E944
:104BB0000201FBF7E7FED4E90201FBF7C5FED4E9E9
:104BC0000201FBF7B3FE606800BF00BF00BF00F149
:104BD000140252E8002F42F0400100F1140242E8B2
:104BE0000013002BF3D100BF00BF606800BF00BFFF
:104BF00000BF00F10C0252E8002F42F0100100F15A
:104C00000C0242E80013002BF3D100BF00BF606824
:104C1000011D0E4632462169A068FBF70FFF226B8B
:104C20002169A068FBF7D0FE2169A068FBF78CFE24
:104C3000606800BF00BF00BF00F1140252E8002FFF
:104C400042F0800100F1140242E80013002BF3D17E
:104C500000BF00BF012084F83800A07D012833D1B7
:104C6000606A68B9218C8800FDF700F96062616AAA
:104C700009B1012100E0002108468221FBF7F2FD85
:104C8000606800BF00BF00BF00F10C0252E8002FB7
:104C900042F4807100F10C0242E80013002BF3D1C2
:104CA00000BF00BF606800BF00BF00BF00F114027A
:104CB00052E8002F42F0010100F1140242E8001313
:104CC000002BF3D100BF00BF70BD7047081C3044FB
:104CD000586C80000000000404040000080000007C
:104CE000080000080000000800020406080A0C0082
:104CF000010203040506081C3044586C80000000C3
:104D0000000404040000080000000800000800007F
:104D1000000800020406080A0C000102030405064C
:104D2000000000000000000001020304060708095B
:104D30000000000001020304081C3044586C80008D
:104D4000000000040404000008000000080000083F
:104D50000000000800020406080A0C000102030417
:104D60000506081C3044586C800000000004040450
:104D70000000080000000800000800000008000211
:104D80000406080A0C000102030405065F6C69733F
:104D900074006C69737420616C6C20636F6D6D615D
:104DA0006E64000000040000000000000800000025
:104DB000080000000020000000000000081C304433
:104DC000586C80000000000404040000080000008B
:104DD000080000080000000800020406080A0C0091
:104DE0000102030405060000000000000000002F7F
:104DF000000000000700070000147F147F14002447
:104E00002A7F2A1200626408132300364955225073
:104E100000000503000000001C22410000004122A8
:104E20001C000014083E08140008083E0808000092
:104E300000A060000008080808080000606000008A
:104E4000002010080402003E5149453E0000427F08
:104E50004000004261514946002141454B31001854
:104E600014127F10002745454539003C4A49493016
:104E700000017109050300364949493600064949D0
:104E8000291E0000363600000000563600000008DB
:104E900014224100001414141414000041221408B8
:104EA00000020151090600324959513E007C12119D
:104EB000127C007F49494936003E41414122007F32
:104EC0004141221C007F49494941007F09090901EC
:104ED000003E4149497A007F0808087F0000417F71
:104EE0004100002040413F01007F08142241007F23
:104EF00040404040007F020C027F007F0408107F8A
:104F0000003E4141413E007F09090906003E4151F2
:104F1000215E007F091929460046494949310001AF
:104F2000017F0101003F4040403F001F2040201F03
:104F3000003F4038403F00631408146300070870C6
:104F4000080700615149454300007F414100005579
:104F50002A552A55000041417F0000040201020445
:104F60000040404040400000010204000020545432
:104F70005478007F48444438003844444420003882
:104F80004444487F00385454541800087E090102F4
:104F90000018A4A4A47C007F080404780000447DC9
:104FA0004000004080847D00007F10284400000005
:104FB000417F4000007C04180478007C08040478D9
:104FC00000384444443800FC2424241800182424C5
:104FD00018FC007C080404080048545454200004C1
:104FE0003F444020003C4040207C001C2040201CCE
:104FF000003C4030403C004428102844001CA0A045
:10500000A07C004464544C44141414141414000080
:105010000000000000000000000000000000000090
:1050200000F8000000000000003330000000001015
:105030000C06100C0600000000000000000040C03C
:105040007840C0784000043F04043F04040000702E
:1050500088FC08300000001820FF211E0000F00826
:10506000F000E018000000211C031E211E0000F0CB
:105070000888700000001E21232419272110101613
:105080000E00000000000000000000000000000012
:1050900000E0180402000000000718204000000291
:1050A0000418E00000000040201807000000404005
:1050B00080F0804040000202010F01020200000067
:1050C00000F0000000000101011F010101000000CB
:1050D00000000000000080B0700000000000000030
:1050E00000000000000000010101010101010000B9
:1050F0000000000000000030300000000000000050
:10510000000080601804006018060100000000E044
:1051100010080810E000000F102020100F000010F1
:1051200010F8000000000020203F20200000007048
:105130000808088870000030282422213000003040
:105140000888884830000018202020110E00000038
:10515000C02010F8000000070424243F240000F8B9
:105160000888880808000019212020110E0000E09E
:10517000108888180000000F112020110E00003840
:105180000808C83808000000003F00000000007058
:10519000880808887000001C222121221C0000E0E1
:1051A00010080810E0000000312222110F0000005A
:1051B00000C0C0000000000000303000000000000F
:1051C000008000000000000080600000000000007F
:1051D0008040201008000001020408102000404018
:1051E000404040404000040404040404040000085B
:1051F0001020408000000020100804020100007010
:1052000048080808F0000000003036010000C030F7
:10521000C828E810E0000718272423140B0000001A
:10522000C038E0000000203C23020227382008F8A4
:10523000888888700000203F202020110E00C03098
:10524000080808083800071820202010080008F86F
:1052500008080810E000203F202020100F0008F868
:105260008888E8081000203F20202320180008F834
:105270008888E8081000203F200003000000C030AC
:1052800008080838000007182020221E020008F82D
:1052900008000008F808203F210101213F200008F4
:1052A00008F8080800000020203F2020000000002F
:1052B0000808F8080800C08080807F00000008F817
:1052C00088C028180800203F20012638200008F850
:1052D000080000000000203F20202020300008F8B7
:1052E000F800F8F80800203F003F003F200008F8D1
:1052F00030C00008F808203F200007183F00E010E9
:1053000008080810E0000F10202020100F0008F8F7
:1053100008080808F000203F210101010000E0100A
:1053200008080810E0000F18242438504F0008F82F
:10533000888888887000203F2000030C302000708F
:105340008808080838000038202121221C0018088D
:1053500008F8080818000000203F2000000008F8A6
:1053600008000008F808001F202020201F000878EF
:10537000880000C83808000007380E010000F8084F
:1053800000F80008F800033C0700073C0300081879
:1053900068808068180820302C03032C30200838DF
:1053A000C800C83808000000203F20000000100896
:1053B0000808C838080020382621202018000000DE
:1053C00000FE020202000000007F40404000000C8E
:1053D00030C000000000000000010638C0000002DC
:1053E0000202FE000000004040407F00000000007C
:1053F000040202020400000000000000000000009F
:10540000000000000000808080808080808000029A
:105410000204000000000000000000000000000086
:105420008080808000000019242222223F2008F87A
:10543000008080000000003F112020110E000000BD
:10544000008080800000000E11202020110000004C
:1054500000808088F800000E112020103F200000FE
:10546000808080800000001F222222221300008002
:1054700080F0888888180020203F2020000000004D
:10548000808080808000006B94949493600008F882
:10549000008080800000203F210000203F2000800D
:1054A0009898000000000020203F2020000000000D
:1054B00000809898000000C08080807F000008F87D
:1054C000000080808000203F24022D302000000852
:1054D00008F8000000000020203F2020000080800D
:1054E000808080808000203F20003F20003F80801F
:1054F000008080800000203F210000203F2000002D
:10550000808080800000001F202020201F008080DD
:1055100000808000000080FFA12020110E0000000C
:10552000008080808000000E112020A0FF808080FD
:1055300080008080800020203F21200001000000AA
:10554000808080808000003324242424190000807F
:1055500080E0808000000000001F2020000080808C
:10556000000000808000001F202020103F2080804D
:1055700080000080808000010E30080601008080DD
:105580000080008080800F300C030C300F00008002
:105590008000808080000020312E0E31200080802D
:1055A00080000080808080818E701806010000805D
:1055B0008080808080000021302C2221300000007B
:1055C0000000807C020200000000003F404000001C
:1055D0000000FF00000000000000FF0000000002CB
:1055E000027C800000000040403F000000000006F8
:1055F000010102020404000000000000000000039A
:10560000050911FF118905C300E000F000F8000052
:1056100000000000004428FF11AA44000000000020
:10562000000000000000000000000000000000007A
:10563000000000000000000000000000000000006A
:10564000000000000000000000000000000000005A
:105650000000000000000000830138448292927430
:105660000183000000000000007C44C7017D7D7DB7
:105670007D017D7D7D7D017D7D7D7D01FF000000C3
:105680000000000100010001000100010001000014
:105690000000000000000001010000000000000008
:1056A00000000000000000000000000000000000FA
:1056B00000000000000000000000000000000000EA
:1056C00000000000000000000000000000000000DA
:1056D00000000000000000000101000000000000C8
:1056E00001010000000000000000000101010101B3
:1056F000010101010101010101010101010000009D
:1057000000000000000000404040404000006D6D7F
:105710006D6D6D0000606060606000004040404062
:105720004000000000000000000000000000000039
:105730000000000000000000000000000000000069
:105740000000000000000000000000000000000059
:105750000000000000000000000000000000000049
:105760000000000000000000000000000000000039
:105770000000000000000000000000000000000029
:1057800000000000000000DBDBDBDBDB0000DBDB1C
:10579000DBDBDB0000DBDBDBDBDB0000DBDBDBDBC5
:1057A000DB0000DADADADADA0000D8D8D8D8D800A4
:1057B00000C0C0C0C0C00000C0C0C0C0C00000C0A9
:1057C000C0C0C0C00000C0C0C0C0C0000080808099
:1057D00080800000000000000000000000000000C9
:1057E00000000000000000000000000000000000B9
:1057F00000000000000000000000000000000000A9
:10580000000000000000000606060606000006066E
:105810000606060000060606060600000606060640
:10582000060000060606E666200006068606060056
:105830000006060606860000060606060600008626
:105840008686868680808686068686C0C086868610
:105850000606D03076060606060000060606060690
:1058600000000606060606000006060606060000FC
:10587000060606060600000000000000000000000A
:105880000000000000000000000000000000000018
:105890000000000000000000000000000000000008
:1058A0000000000000000000601C00FE000102007B
:1058B000C41820029E63B20E00FF8181FF000080A9
:1058C00040300F00000000FF0023EAAABFAAEA034D
:1058D0003F00FF000000000000000000000000008A
:1058E00000000000000000000000000000000000B8
:1058F00000000000000000000000000000000000A8
:105900000080808000000000008080800000000097
:105910000000000000000000000000000000000087
:105920000000000000000E0C080000010101010150
:1059300000000001000000010081808081808180E2
:1059400080808001010101000000010000000100D1
:105950000101090C0E000000000000000000000022
:10596000000000000000C0C0C0C0C0C0C0C0C0C0B7
:10597000C0C0C0C0C0C0C0C0C0C0C0C0C000001E49
:1059800021404050215E001E21404050215E000019
:105990000000000000000000000000000000000007
:1059A00000000000000000000000000000000000F7
:1059B000000000000000000000FFFFC1C1FFFFC1A8
:1059C000C1FFFF0000000000000000000000000018
:1059D00000000000000000000000000000000000C7
:1059E000000000000000FFFF80FCF3EFF3FC80FFED
:1059F00080EEEEEEF5FBFF9CBEB6B688FF00000021
:105A0000205A000800000020700000001C1D000843
:105A1000905A000870000020903400002C1D0008EF
:105A20000024F4000000000000000000000000005E
:105A30000000000000000000000000000000000066
:105A40000000000000000000000000000000000056
:105A5000000000000000000000000000B92E000857
:105A6000A52F00088000002000C001208020002019
:105A700038000020000000000000000000000000CE
:105A80008C4D0008924D0008C6E533B4491E00084D
:04000005080000ED02
:00000001FF
